:100000000C94ED020C9425030C9425030C94250309
:100010000C9425030C9425030C9425030C942503C0
:100020000C9425030C9425030C94B9190C94F51821
:100030000C942E120C9425030C9425030C94250388
:100040000C9425030C9425030C9425030C94250390
:100050000C9425030C94ED110C9425030C942503AA
:100060000C9425030C9425030C9425030C94250370
:100070000C9425030C9425030C9425030C94250360
:100080000C9425030C9425030C9425030C94250350
:100090000C9425030C9425030C9425030C94250340
:1000A0000C9425030C9425030C9425035107510748
:1000B00083078307F5071108A809A8091C08FA088F
:1000C0000B090B0903172A17CD182A17CD18721719
:1000D0009517CD1884189818000000000000000043
:1000E0000000000000000000000000000000000010
:1000F0000000000000000000000000007E0F00D49F
:10010000FFFFFFC7000000780000000000000000B3
:100110002A2B280000000000000000000000000062
:1001200000000029000000002C1E3420212224346D
:100130002627252E362D3738271E1F20212223243F
:1001400025263333362E37381F0405060708090ADB
:100150000B0C0D0E0F101112131415161718191A77
:100160001B1C1D2F3130232D350405060708090AF5
:100170000B0C0D0E0F101112131415161718191A57
:100180001B1C1D2F3130354C68747470733A2F2F3F
:10019000716D6B2E666D2F0A00514D4B20697320D7
:1001A0007468652062657374207468696E67206581
:1001B000766572210000047F3F1F6432146432149C
:1001C000783C1E1E140A052223252628292A2C2DB8
:1001D0002F3032333536383A3B3D3E404243454777
:1001E000494A4C4E5051535557595A5C5E606264AF
:1001F0006668696B6D6F71737577797B7D7F8183BD
:100200008587898A8C8E90929496989A9C9E9FA1BD
:10021000A3A5A7A8AAACAEAFB1B3B4B6B8B9BBBCDE
:10022000BEBFC1C2C3C5C6C7C9CACBCCCDCED0D153
:10023000D2D2D3D4D5D6D7D7D8D9D9DADADBDBDB4B
:10024000DCDCDCDCDCDDDDDDDDDCDCDCDCDCDBDBEC
:10025000DBDADAD9D9D8D7D7D6D5D4D3D2D2D1D040
:10026000CECDCCCBCAC9C7C6C5C3C2C1BFBEBCBB3D
:10027000B9B8B6B4B3B1AFAEACAAA8A7A5A3A19FB5
:100280009E9C9A98969492908E8C8A898785838179
:100290007F7D7B79777573716F6D6B69686664625A
:1002A000605E5C5A5957555351504E4C4A49474528
:1002B0004342403E3D3B3A3836353332302F2D2CC9
:1002C0002A29282625232205010902A101850209E0
:1002D00001A10005091901290815002501950875D6
:1002E0000181020501093009311581257F950275CB
:1002F00008810609381581257F9501750881060555
:100300000C0A38021581257F950175088106C0C049
:1003100005010980A101850319012AB700150126ED
:10032000B700950175108100C0050C0901A1018578
:100330000419012AA002150126A002950175108159
:1003400000C005010906A1018506050719E029E796
:10035000150025019508750181020507190029EF8F
:100360001500250195F0750181020508190129057F
:10037000950575019102950175039101C00501096B
:1003800006A101050719E029E71500250195087563
:100390000181029501750881010507190029FF15E2
:1003A0000026FF009506750881000508190129053A
:1003B000950575019102950175039101C009029F90
:1003C00000040100A0FA0904000001030101000972
:1003D00021110100012240000705810308000109E5
:1003E000040100010300000009211101000122B6EF
:1003F0000007058203200001080B02020101000032
:1004000009040200000101000009240100010900A3
:100410000103090403000201030000072401000195
:100420004100062402010100062402020200092400
:100430000301030102010009240302040101010078
:100440000905040240000500000525010101090518
:10045000830240000500000525010103120100028E
:1004600000000008A80300000100010200011A03B7
:100470006E0061006E006F002E00200073006C00A3
:100480006900640065007200000014036B006500E1
:10049000650062007700650072006B002E000000AE
:1004A0000403090420002100220023001F00115032
:1004B0001E002700CA5CA85DC55CCB5CC45C125002
:1004C000C35CA75D7300BC00BB007200A9001050A4
:1004D000AA00AE00000101010101010101010202B7
:1004E00002020202020202030303030303030304E2
:1004F00004040404040405050505050606060606AD
:10050000070707070708080808090909090A0A0A66
:100510000B0B0B0C0C0C0D0D0D0E0E0E0F0F0F1008
:100520001011111112121313141415151616171792
:10053000181819191A1A1B1B1C1D1D1E1E1F2020FE
:10054000212222232424252626272829292A2B2C48
:100550002D2D2E2F30313232333435363738393A6B
:100560003B3C3D3E3F404142434445464748494A63
:100570004C4D4E4F50515354555658595A5B5D5E31
:100580005F616264656668696B6C6D6F70727375CC
:1005900077787A7B7D7E8082838587888A8C8E8F30
:1005A00091939596989A9C9EA0A2A3A5A7A9ABAD5E
:1005B000AFB1B3B5B7BABCBEC0C2C4C6C9CBCDCF4C
:1005C000D1D4D6D8DBDDDFE2E4E7E9EBEEF0F3F5FA
:1005D000F8FAFDFFFFAA7F55400011241FBECFEFA0
:1005E000DAE0DEBFCDBF04B603FE18C080918503FC
:1005F00090918603A0918703B09188038730904B38
:10060000A740B04B59F410928503109286031092C4
:10061000870310928803E0E0F8E3099511E0A0E079
:10062000B1E0EEE2F2E502C005900D92A239B10709
:10063000D9F723E0A2E9B1E001C01D92A538B207C5
:10064000E1F70E94E70A0C9415290C940000AF9280
:10065000BF92CF92DF92EF92FF920F931F93CF93AF
:10066000DF93EC018AE0A82EFE012491222309F4F5
:1006700095C0213009F03DC031968491813021F43C
:100680002296FE01849184C0823031F42296FE01CC
:1006900084910E94461E80C0833031F42296FE0170
:1006A00084910E94E61D78C0843009F074C02296BF
:1006B000FE01249180E090E030E0205331092A309F
:1006C000310560F4A89EA001A99E500D1124C90116
:1006D000840F951F2196FE012491EECF009709F417
:1006E0005BC0EFE9FFE03197F1F700C00000019730
:1006F000F5CFE22FF0E0E85FFE4FB490822F8695B1
:100700008695869590E0FC01E850FF4FE4902770B5
:10071000F12C022E02C0F594E7940A94E2F7F1E07E
:10072000EF22FF24FC01E851FF4FC490D12C022E90
:1007300002C0D594C7940A94E2F731E0C322DD24C5
:10074000FC01E852FF4F049110E002C01595079597
:100750002A95E2F701701127E114F10419F081EEF6
:100760000E94461EC114D10419F086EE0E94461E56
:100770008B2D0E940A1FCD2819F086EE0E94E61DDF
:10078000EF2819F081EE0E94E61D012B29F08CE282
:100790000E940A1F01C0EF01219666CFDF91CF9121
:1007A0001F910F91FF90EF90DF90CF90BF90AF908F
:1007B00008951F93CF93DF93CDB7DEB767970FB63A
:1007C000F894DEBF0FBECDBF4B8B5C8B6D8B7E8BE9
:1007D0008F8B61111092800286E09E01235F3F4F54
:1007E000D901E82F1D92EA95E9F795E0FE0173968D
:1007F000D90101900D929A95E1F79C894E895F8904
:100800007B897D879E876F87598B488BF901DE0135
:10081000179601900D928A95E1F7CE0107960E94F6
:10082000701B81113EC086E0FE013796DE011196F5
:1008300001900D928A95E1F7FF81E8856A857B85B5
:100840006115710531F0EF3F31F481E0FF3F19F49C
:1008500003C081E001C080E080FD23C020912D0213
:1008600030E0C90101968770992740915E0250E0FF
:100870008417950779F1F983EA837D836C8396E089
:10088000929FD001939FB00D1124A25DBD4FFE0138
:10089000319601900D929A95E1F780932D020E9476
:1008A000192316E080915E0290912D028917F9F0CC
:1008B000189FC0011124825D9D4F0E94701B8823E8
:1008C000B1F080915E0290E0019687709927809345
:1008D0005E02E8CF0E94C01D10922D0210925E02AF
:1008E000E7E2F2E086E0DF011D928A95E9F767967C
:1008F0000FB6F894DEBF0FBECDBFDF91CF911F9131
:1009000008958F929F92AF92BF92CF92DF92EF9213
:10091000FF920F931F93CF93DF93CDB7DEB72A9744
:100920000FB6F894DEBF0FBECDBFFC01D0801181A1
:1009300083819481892B39F01F3F39F491E00FEFC7
:10094000D01203C003C091E001C090E090FD2CC61E
:100950007F0185E0DE01169601900D928A95E1F700
:10096000F70122818E819F81222349F00E94DE1AA5
:10097000082F682F8E819F810E943C1D03C00E941A
:10098000111D082FE12FF0E0E00FF11DE00FF11D28
:10099000EE0FFF1FEE0FFF1FED0DF11DEE0FFF1FFE
:1009A000EC55FB4F05911491073AFDE51F0729F01F
:1009B000083A2DE5120749F012C0F7018281882319
:1009C00009F454C089E991E007C0F70182818823C6
:1009D00009F44CC088E891E00E94270347C0043F17
:1009E000FCE51F0759F190F4093D3CE51307E9F0D8
:1009F0000A3D8CE51807A1F1083D9CE51907B1F502
:100A000006E221EE41EE68ED7CE514C0063FECE520
:100A10001E0701F1C8F0073F2CE5120739F507E280
:100A200025EE46EE67EF7CE505C007E225EE45EED4
:100A300069ED7CE5C7010E94EC12DFC406E221EEFD
:100A400040EE64EF7CE5F6CF07E225EE44EE65EF7D
:100A50007CE5F0CF06E221EE42EE66EF7CE5EACFE0
:100A600008E221E045EE6AED7CE5E4CFF701828102
:100A7000882309F45BC11092C2010430FDE51F0711
:100A800058F40B3F2CE5120780F4C80182509C45B6
:100A9000449708F035C109C002363DE5130729F037
:100AA000063A8DE5180709F02BC10E9401229093A8
:100AB000CF018093CE0101319CE5190709F4C6C02E
:100AC00008F042C00930FCE51F0709F49BC000F59F
:100AD00005303CE5130709F485C078F403309CE544
:100AE000190709F478C008F07AC002301C4509F0F3
:100AF000F7C08091CE018160F1C007302CE512076C
:100B000009F478C008F07AC08091CE018061E6C017
:100B10000D308CE5180709F487C058F40B30ECE56C
:100B20001E0709F479C008F07BC08091CE0188606F
:100B30006FC00F302CE5120709F480C008F082C0A6
:100B40008091CE01877FCAC00E3F8CE5180709F45B
:100B500071C000F50531ECE51E0709F485C068F4A5
:100B600003312CE5120709F475C008F095C00E9406
:100B7000C01D8091CE018F77B1C00C3F8CE5180766
:100B8000A9F108F054C00B3F1C4509F0A9C08091A1
:100B9000CF0140C00230FDE51F0709F489C058F4B9
:100BA00001153DE5130709F45AC008F069C08091AA
:100BB000CF0182602FC002369DE5190709F47EC07F
:100BC000063AEDE51E0709F483C003301D4509F020
:100BD00087C060E06EC08091CE0182607FC080914E
:100BE000CE0116C08091CE01886078C08091CF017F
:100BF00082604FC08091CE01806270C08091CE0132
:100C000080646CC00E94C01D8091CE01806866C067
:100C1000846064C081603DC08091CE018E7F5EC0E3
:100C20008091CE018D7F5AC08091CE0116C08091F7
:100C3000CF0118C08091CF018D7F2BC08091CE0154
:100C40008F7E4CC08091CE018F7D48C08091CE01B7
:100C50008F7B44C08091CE01877F8B7F3FC0809186
:100C6000CF018D7F8E7F15C08091CE0182FB222720
:100C700020F991E0922790FB82F990FB83F92EC036
:100C80008091CF01982F909591708E7F892B90FB4A
:100C900081F98093CF0124C00E94C01D8091CE01B4
:100CA00087FB222720F991E0922790FB87F916C055
:100CB00061E08EE090E00E94462812C08091CE0153
:100CC00084FB222720F991E0922790FB84F906C04B
:100CD0008091CE01982F909590FB80F98093CE0162
:100CE0006091CE011091CF0184E090E00E944628EF
:100CF000612F82E290E00E9446280E94C01D7DC3C1
:100D00000631FCE51F0721F5809181028A7A91E086
:100D100009F490E090939401882311F065E301C0F9
:100D200069E287E092E00E947F120FC00631FCE585
:100D30001F0709F040C080919401882309F480C303
:100D400065E387E092E00E9457120E948A2255C311
:100D50000B353DE5130749F158F401159CE51907DA
:100D6000B1F00F3D1C4509F042C00E94122245C35C
:100D70000C35FDE51F07D9F00D351D45C1F58091F6
:100D8000CF0182FB882780F991E0892711C00E945A
:100D9000C01D3FEF84E39CE0315080409040E1F77C
:100DA00000C000000E94C91128C381E001C080E09A
:100DB0000E94FC221CC08091810282720D3C2CE5B5
:100DC000120709F4D1C308F001C3073C9CE51907D9
:100DD00009F4B6C308F044C3043CFCE51F0709F45A
:100DE000A5C308F02FC3033C1C4509F47AC3F701DF
:100DF000828100811181882349F0C8010E94DE1A96
:100E0000D82E682FC8010E943C1D04C0C8010E9452
:100E1000111DD82EE12FF0E0ED0DF11DED0DF11DAE
:100E2000EE0FFF1FEE0FFF1FE00FF11DEE0FFF1F74
:100E3000EC55FB4F859194910E9467208C01982E70
:100E4000F701D280A580A2946FE0A62280915F0274
:100E50008770B9F0DD20A9F0812F807F803421F0E8
:100E600080E2800F883068F08091CF0182FD09C058
:100E700082E00E94DF2280915F028770CC24C394BD
:100E80008111C12CB12EB2943FE0B3228B2D90E0A2
:100E90008C30910508F05CC2FC01EA5AFF4F0C94BB
:100EA000C428812F807F1F70882311F01295107F36
:100EB000DD20B9F0112309F438C280E2800F8830B8
:100EC00010F0911006C080918102182B10938102BE
:100ED00005C080918002182B109380020E948A2204
:100EE00024C2802F0E94E61D112309F431C2005E46
:100EF000083078F1992069F11095809180021823CB
:100F00001093800229C0812F807F1F70803211F0E2
:100F10001295107F992021F0F1E09F16D9F149C078
:100F20008091CF0182FF1BC0DD2069F0112339F0D1
:100F300080918102182B109381020E948A2280E006
:100F40000E94461E05C280E00E94E61D112309F49E
:100F5000FFC1812F0E9483220E948A22F9C1DD20D5
:100F600081F080918202AA2051F001E0A01207C016
:100F7000182B181709F4ECC110938202E9C1812BD8
:100F800010C0AA2021F021E0A21609F4E1C10E94BC
:100F90007D2227C0DD2041F035E03A1508F4D8C1A4
:100FA000812F0E94DC1DD4C184E08A1508F4D0C1D1
:100FB00018C0DD2049F0AA2099F3F701858180FF50
:100FC000B4C18F708583ECCFAA2059F0093309F0A2
:100FD000BCC1FFEF17EE23E0F15010402040E1F7D5
:100FE000B2C1812F0E94D51DB3C1812F86958695F0
:100FF000837019F0813059F0ABC1DD2019F0C801C0
:10100000937002C080E090E00E94CA12A7C1DD2068
:1010100019F0C801937002C080E090E00E94B41201
:101020009DC1802FDD2019F00E94AF2602C00E94D2
:10103000F6250E94CC2592C1812F837009F069C0EA
:10104000D1108AC1902F929596959770990F990F0C
:10105000802F8F70882E912CA12CB12C092E04C0CA
:10106000880C991CAA1CBB1C0A94D2F704FF12C05E
:101070004FE050E060E070E004C0440F551F661F71
:10108000771F9A95D2F7DB01CA0180959095A095BC
:10109000B09503C080E090E0DC0116951695412FD5
:1010A0004370423019F1C8F4009183021091840218
:1010B0002091850230918602413059F08829992982
:1010C000AA29BB29BC01CD0160237123822393236C
:1010D0000AC0802A912AA22AB32ABC01CD0168291C
:1010E00079298A299B290E94B61D36C18829992908
:1010F000AA29BB29009183021091840220918502C4
:1011000030918602BC01CD01602771278227932789
:10111000EACFDD2019F0812F817001C086958823E8
:1011200009F41AC1902F929596959770990F990F7F
:10113000802F8F70882E912CA12CB12C092E04C0E9
:10114000880C991CAA1CBB1C0A94D2F704FF12C07D
:101150004FE050E060E070E004C0440F551F661F90
:10116000771F9A95D2F7DB01CA0180959095A095DB
:10117000B09503C080E090E0DC0116951695412FF4
:1011800043704230D9F068F50091970110919801B1
:101190002091990130919A01413059F0882999297B
:1011A000AA29BB29BC01CD0160237123822393238B
:1011B0001EC0802A912AA22AB32A13C088299929FD
:1011C000AA29BB29009197011091980120919901BA
:1011D00030919A01BC01CD016027712782279327A6
:1011E00006C0BC01CD01682979298A299B290E9462
:1011F000661DB2C01F70DD2039F0812F0E94951D41
:10120000802F0E94DC1DA8C0802F0E94D51D812F39
:101210000E94701DA1C0802F32EF931609F443C0C5
:10122000391538F090EF991659F0E1EF9E16B1F1AB
:1012300077C0F3EF9F16F1F124EF921659F170C0C9
:10124000DD2019F134E03A1508F482C01F7181E005
:1012500090E0A0E0B0E0AC01BD0104C0440F551F18
:10126000661F771F1A95D2F7809197019091980188
:10127000A0919901B0919A018A019B010827192731
:101280002A273B27C901B80129C025E02A1508F4FF
:101290005FC0DCCF8091CF0182FF23C0DD2029F029
:1012A000812F8F7130C0DD20D9F3812F8F710E9483
:1012B000701D4EC0DD2079F01F7181E090E0A0E04C
:1012C000B0E0BC01CD0104C0660F771F881F991FD5
:1012D0001A95D2F703C060E070E0CB010E94661D52
:1012E00037C0DD2099F01F71812F0E94951D8091DC
:1012F000CF0182FD07C038E0139FC0011124836035
:1013000080935F02812F0E94951D22C081E00E9480
:10131000DF2281E08A15E0F482E00E94DF2218C01B
:10132000DD2029F0AA2009F4BBCF802F09CEAA2006
:1013300009F4BBCF893349F49FEFE7EEF3E0915016
:10134000E040F040E1F700C00000802F0E94E61D61
:1013500088EF8B0D843010F40E94E012CC20A9F0AD
:1013600080915F0280FD11C0F701128285958595FD
:1013700085950E94951DC7010E94810480915F029E
:101380008595859585950E94701D85E0F701DE01A4
:10139000119601900D928A95E1F789819A810E94B8
:1013A000111DE82FF0E0EE0FFF1F8A81E80FF11DFD
:1013B000EE0FFF1FEE0FFF1F8981E80FF11DEE0FEB
:1013C000FF1FEC55FB4F85919491EEC0023D2CE53B
:1013D000120709F4D9C008F465C0053D2CE51207D1
:1013E00009F4D8C008F471C0063DECE51E0709F405
:1013F000D6C00E351D4509F0FACC80915F0287708A
:1014000009F4D2C0F7018281882309F4CDC080910C
:10141000CF0182FDC9C082E02A960FB6F894DEBFE4
:101420000FBECDBFDF91CF911F910F91FF90EF9035
:10143000DF90CF90BF90AF909F908F900C94DF2261
:1014400069E27FCC053C9CE5190709F474C0063CB1
:101450001C4509F0CCCC4CE655E265E775E288C046
:101460000A3CFCE51F0709F475C070F4083C3CE534
:10147000130709F46AC0093C1C4509F0B8CC40E6E2
:1014800055E264E575E274C00B3CECE51E0709F417
:1014900066C00C3C1C4509F0AACC45EC53E266ED55
:1014A00073E266C00F3C8CE5180709F467C008F4C6
:1014B00062C0003DECE51E0709F463C0013D1C4518
:1014C00009F095CC6EE089E067C0033D8CE5180714
:1014D00009F45DC0043D1C4509F089CC61E088E158
:1014E00060C08091BB0180FF1BC08E7F8093BB01D9
:1014F0006091BB017091BC018091BD019091BE01D2
:101500000E94B3231092AB010FEF10E722E00150CD
:1015100010402040E1F700C000000E948D136DCF05
:1015200081608093BB0161E086953BC049EB55E249
:1015300062EC75E21DC042EC55E269EB75E218C041
:1015400045E755E26CE675E213C044E555E260E616
:1015500075E20EC04CE355E268E475E209C048E468
:1015600055E26CE375E204C046ED53E265EC73E2CC
:101570000E94711342CF61E081E013C065E082E018
:101580000BC068E086E008C064E18FE005C067E159
:1015900085E102C062E289E10E945F132ECF61E023
:1015A00083E20E947E2529CF2A960FB6F894DEBFEB
:1015B0000FBECDBFDF91CF911F910F91FF90EF90A4
:1015C000DF90CF90BF90AF909F908F900895CF9372
:1015D000DF93CDB7DEB760970FB6F894DEBF0FBECE
:1015E000CDBF1092BD021092BF021092BE0280ECDD
:1015F0008093820380EC92E0909384038093830332
:10160000109281031092800310929D0210929C020E
:1016100010929F0210929E021092A1021092A002BC
:101620001092A3021092A2021092A5021092A4029C
:101630001092A7021092A6021092A9021092A8027C
:101640001092AB021092AA021092AD021092AC025C
:101650001092AF021092AE021092B1021092B0023C
:101660001092B3021092B2021092B7021092B60218
:101670008CE691E1909399028093980288EB90E137
:101680009093B9028093B80281EA9FE09093B502EB
:101690008093B40280EA9FE090939B0280939A0229
:1016A00084B7877F84BF0FB6F894A89580916000B7
:1016B000886180936000109260000FBE90E080E827
:1016C0000FB6F89480936100909361000FBE85B7C8
:1016D000806885BF85B7806885BF88E29FE1909369
:1016E0009301809392010E9439190E9458198091A8
:1016F000E20084608093E20078948091F80188236E
:10170000A1F01091E9001F709091EC00892F817079
:1017100090FD80E8182B1092E9008091E80083FD8D
:101720000E941E161F701093E90082E084BD93E0B2
:1017300095BD9AEF97BD80936E0080EF0E946D1F5C
:1017400081EF0E946D1F09E211E08DE2E82E81E039
:10175000F82EF80181918F018F3F11F00E946D1FCB
:10176000E016F106B1F710929F0110929E011092BF
:1017700096011092950180E090E00E944028893EF9
:101780009E4F11F00E94122282E090E00E943228C7
:101790008093A0010E9401229093CF018093CE01FB
:1017A0000E94841F8FE39CE90197F1F700C00000BD
:1017B0000E94841F80919E0180FF08C06FEF7FEF21
:1017C00080E090E00E9464280E94C91183E090E0CC
:1017D0000E943228682F70E080E090E00E94B61DE1
:1017E00080919B01811136C080E090E00E944028EA
:1017F000893E9E4F21F00E9412220E94E72388E03A
:1018000090E00E943A286093BB017093BC018093E2
:10181000BD019093BE016E7F71F40E94E72388E0C2
:1018200090E00E943A286093BB017093BC018093C2
:10183000BD019093BE010E94A0231092AB01809144
:10184000BB0180FF04C060E086950E947E2581E098
:1018500080939B0180E091E09093C6018093C50145
:1018600018E1812E912C00E4E02EFF24F3945524FE
:1018700053948091F801853009F06FC000E112E1C6
:101880008091F801853009F053C08091F8018430CF
:1018900009F43DC01092AB0180919D01811116C0E9
:1018A00050929D018091BB01982F917090939C0163
:1018B0008E7F8093BB01FFEF20E732E0F1502040A4
:1018C0003040E1F700C000000E948D131092C90162
:1018D0000FB6F894A895809260000FBEE092600069
:1018E00083B7817F846083BF83B7816083BF78942F
:1018F000889583B78E7F83BF0FB6F894A8958091A3
:101900006000886180936000109260000FBE80913B
:10191000F701882309F4B4CF0E94841F80919E01AF
:101920008111EBC280919F01882309F4A9CFE5C200
:101930000E94C01D0E94E01210929D0180919C01A6
:10194000882349F08091BB0181608093BB0160E0F6
:1019500086950E947E250E9477130E94841F88230B
:1019600059F08FB7F8944091CA015091CB01609122
:10197000CC017091CD018FBFAEE9B1E0E1EAF1E0B9
:1019800000E010E0302F2D919191922721F180E01D
:10199000DD24D394492F4D21D1F08F8338872D2119
:1019A00081E009F480E089870E9422128160782F0B
:1019B0009B878A874F81588569858B850E94D903CB
:1019C000F801EF55FE4F8081D826D08219C08F5F75
:1019D000DD0C8430F9F60F5F1F4F0230110591F6D0
:1019E0008FEF8C878D871E860E9422128160782F50
:1019F000988B8F874C855D856E8588890E94D90379
:101A00008091AB01882309F493C08091AA01E091F1
:101A1000BB01E695E81BE093A601823059F4F0E0A3
:101A2000ED53FE4FE4910E2F10E0B3E5CB2EB0E165
:101A3000DB2E59C0863059F4F0E0E054FE4FE491BB
:101A40000E2F10E0A3E4CA2EA0E1DA2E4CC089309C
:101A500061F4E695F0E0E354FE4FE4910E2F10E0C0
:101A6000F9E3CF2EF5E1DF2E3EC08F3061F4E6952D
:101A7000F0E0E654FE4FE4910E2F10E0E5EDCE2E9F
:101A8000E4E1DE2E30C0853159F4F0E0E954FE4F38
:101A9000E4910E2F10E077E8C72E74E1D72E23C013
:101AA0008831A1F0833249F4E5EBF1E0059114911E
:101AB00063E0C62E60E1D62E16C0843271F404EFC6
:101AC00011E053ECC52E53E1D52E0DC008E210E015
:101AD0004DEFC42E43E1D42E06C000ED17E032EAEC
:101AE000C32E3FE0D32E8091A701882361F010928E
:101AF000A7010E9422129093A5018093A401109245
:101B0000A9011092A8010E942212E091A401F09173
:101B1000A5018E1B9F0B8F3F9F4750F40E0F1F1F79
:101B20001093A5010093A40184EA91E0F6010995C0
:101B300086E0E2E9F2E0DE01119601900D928A95CD
:101B4000E1F7C0909402D090950200919602109116
:101B5000970210929402109295021092960210929F
:101B60009702C11003C0DD2009F44FC0809190029C
:101B7000909191020E9413129C0190918C029923E2
:101B800009F4D1C12531310508F43FC09F3F19F058
:101B90009F5F90938C02CC2061F00E948F261C14D2
:101BA00014F09FEF01C091E0899F802D1124809354
:101BB0009402DD2061F00E948F261D1414F09FEF27
:101BC00001C091E0899F802D11248093950230916E
:101BD00094023323D1F0209195022223B1F045EBFA
:101BE0003403C0011124992319F09093940202C088
:101BF000F092940235EB2303C0011124992319F0CC
:101C00009093950202C0F0929502011103C0112336
:101C100009F44FC080918E0290918F020E9413129E
:101C20009C0190918B02992309F482C121353105E1
:101C300008F43FC09F3F19F09F5F90938B020023F1
:101C400061F00E946D26101614F09FEF01C091E024
:101C5000899F802D112480939602112361F00E94A8
:101C60006D26111614F09FEF01C091E0899F802D21
:101C7000112480939702309196023323D1F0209162
:101C800097022223B1F045EB3403C00111249923BC
:101C900019F09093960202C0F092960235EB23035E
:101CA000C0011124992319F09093970202C0F09279
:101CB00097028091940281110BC08091950281114D
:101CC00007C080919602811103C080919702811113
:101CD0000E94CC25CB82DC820D831E8386E0FE0130
:101CE0003196A2E9B2E001900D928A95E1F7E09178
:101CF000B802F091B902309719F088E992E009959D
:101D00002FB7F8940091810390918003091718F47C
:101D100080918203080F091B2FBFC12CD12C10E02A
:101D200083E0682E712CAA24A394B12C24E0322ED7
:101D3000C016D10608F0B4C08091800390E0609195
:101D4000820370E00E948E28E0918303F091840367
:101D5000E80FF91F40802090BD0247EF441560F462
:101D6000F092BD0220E040E0642D81E090E00E940E
:101D70000A272092BD0282C047FE4FC084E0281689
:101D800031F04092BA02B092BF02A092BE02842DFE
:101D90000E949210813031F080F0823059F083300F
:101DA00049F034C08093BD0220E040E0642D81E022
:101DB00090E027C08093BD0261C090EF4916E1F02A
:101DC000E7EF4E1223C02091BE023091BF02C9013D
:101DD000B3010E947A28FC01E856FD4F42A2C901D6
:101DE00001969093BF028093BE022091BC02409165
:101DF000BB026091BA0205C03092BD024092BA02A5
:101E000033C00E940A271092BD0238C01092BD0252
:101E10001092BF021092BE0231C0222079F12091AF
:101E2000BE023091BF02C901B3010E947A28AC0101
:101E3000FC01E856FD4F42A2C90101969093BF02F2
:101E40008093BE0241305105A1F042305105B1F4FA
:101E50002091BC024091BB026091BA020E940A2705
:101E60008091BD02843051F0B092BF02A092BE02B8
:101E700005C0F2E02F1202C020E0ECCF2FB7F8949B
:101E80008091800390E001966091820370E00E944F
:101E90008E28809380032FBF2FEFC21AD20A48CF1B
:101EA0000E94E0129091A30189138093A301809175
:101EB000F801843009F0DDCC80911B018F70809394
:101EC000E9009091E80090FFD4CC9091F801943013
:101ED00009F0CFCC8093E9002091F3008091F200CB
:101EE00090E0922B892B09F4C4CC8091E8008E7786
:101EF0008093E8000E94901ABCCC09BD19BD09B4BA
:101F000000FEFDCF8091D8008F7D8093D800809116
:101F1000E00082608093E0008091E00081FDFCCFD2
:101F20000E94C01DADCC2B30310508F031CE6DCEF6
:101F30002B30310508F080CEBCCE8091D5010895BC
:101F400008950895089522E02093E9002FEF30913D
:101F5000E800215035FD06C035ED3A95F1F7000057
:101F60002111F5CF2091E80025FF0BC040E050E0A3
:101F700066E070E00E9406288091E8008E778093EA
:101F8000E8000895CF93DF9320912601222339F0B2
:101F90002091CE0127FF03C060E222E002C068E08A
:101FA00021E02093E9002FEF3091E800215035FD2A
:101FB00006C035ED3A95F1F700002111F5CF2091DB
:101FC000E80025FF1DC0EC0180912601811105C0AC
:101FD00040E050E068E070E003C070E040E050E0B6
:101FE000CE010E9406288091E8008E778093E80059
:101FF00080E2FE01A6EDB1E001900D928A95E1F735
:10200000DF91CF9108950F931F93CF93DF9300D06B
:102010001F92CDB7DEB78C018091AE0181110AC04D
:102020009E012F5F3F4F4FEF6FEF0E94F6238A8193
:102030008093AE01F8018481813051F028F0823024
:1020400061F44091AE010AC08091AE0140E007C04A
:102050006091AE0140E080E003C040E080E060E0DD
:102060000E948F23F801848190E0019663E070E084
:102070000E948E2884830F900F900F90DF91CF9154
:102080001F910F910895CF93DF93EC01EBEBF1E0FB
:10209000438162818C810E948C248C818F5F8C8330
:1020A000DF91CF910895CF93DF93EC01EC81F0E0C5
:1020B000E953FE4F4491EBEBF1E0628181810E9494
:1020C0008C248C818F5F8C83DF91CF9108958093D6
:1020D000D0017093D2016093D1018091F8018430D6
:1020E00001F582E08093E9008FEF9091E800815044
:1020F00095FD06C095ED9A95F1F700008111F5CF99
:102100008091E80085FF0DC040E050E063E070E0A2
:1021100080ED91E00E9406288091E8008E77809300
:10212000E8000895982F907F903BF1F038F49039B3
:10213000D9F0903AC9F09038C9F416C0903D49F0F2
:1021400018F4903C31F012C0903E71F0903F19F0BD
:102150000DC082E00895815F8F3040F4E82FF0E0F9
:10216000E35DFE4F8081089583E0089580E0089547
:10217000AF92BF92CF92DF92EF92FF920F931F9395
:10218000CF93DF93CDB7DEB727970FB6F894DEBFB6
:102190000FBECDBF7E0125E0E20EF11C8C0108517F
:1021A0001F4F8091F801843009F085C08091200193
:1021B0008F708093E9008091E80082FF7CC080915D
:1021C000E80085FF78C00E94901A81111DC084E04C
:1021D000C82ED12CCE0101965C0109C08091F1007E
:1021E000D5018D935D01B1E0CB1AD10869F08091E2
:1021F000E80085FDF3CF8091E8008B778093E800BD
:102200000E94901A882399F38091E80085FD05C00B
:102210008091E8008B778093E800DA808D2D0E9412
:102220009210282FDD828B818E838C818F832111E8
:102230000FC08981843049F0873039F0863039F019
:10224000853009F0AECF21E003C023E001C022E0D9
:1022500067018C2D8E19821708F0A3CFD601BD908F
:102260006D013FB7F894D8011196EC911197F0E009
:10227000CF01019612966C9170E00E948E28D801D1
:102280004C9150E084179507A1F0D80113968D91D9
:102290009C911497E80FF91FB08211968C911197B9
:1022A00090E0019612966C9170E00E948E28F801E1
:1022B00081833FBFCECF27960FB6F894DEBF0FBE07
:1022C000CDBFDF91CF911F910F91FF90EF90DF90E5
:1022D000CF90BF90AF900895DF92EF92FF920F934F
:1022E0001F93CF93DF9300D000D0CDB7DEB77B0133
:1022F000142FD22E4A832B830C83842F0E9492109A
:1023000081111CC082E0E816F10471F083E0E81648
:10231000F10421F0EA94EF2881F50BC0073F11F496
:1023200087E00AC084E008C087EFD812FBCF86E0C0
:1023300003C0173FB9F785E0898303C012951F706A
:1023400019838091F8018430C1F480911B018F7052
:102350008093E90040E050E064E070E0CE01019637
:102360000E940628811109C08091E80085FD05C002
:102370008091E8008E778093E8000F900F900F9087
:102380000F90DF91CF911F910F91FF90EF90DF9011
:10239000089581E08093E00080E28093D80010925D
:1023A000C9008FE19EE40197F1F700C0000087E0CB
:1023B00090EBDC018093850390938603A0938703C1
:1023C000B09388039CE088E10FB6F894A8958093B9
:1023D00060000FBE90936000FFCF78941F920F9221
:1023E0000FB60F9211248F939F93AF93BF93809159
:1023F000CA019091CB01A091CC01B091CD01019681
:10240000A11DB11D8093CA019093CB01A093CC0173
:10241000B093CD01BF91AF919F918F910F900FBE5F
:102420000F901F9018959C014FB7F8948091CA01A6
:102430009091CB01A091CC01B091CD014FBF821BF7
:10244000930B08952FB7F8948091CA019091CB0116
:10245000A091CC01B091CD012FBF08951F920F9292
:102460000FB60F9211248F939F93AF93BF938091D8
:10247000C901811113C08091CA019091CB01A09133
:10248000CC01B091CD014196A11DB11D8093CA012F
:102490009093CB01A093CC01B093CD01BF91AF91AC
:1024A0009F918F910F900FBE0F901F9018952091C4
:1024B00026012223C9F02091CE0127FF15C0262F27
:1024C0002695269526952E31C8F4FC01E20FF11DC4
:1024D000677081E090E001C0880F6A95EAF7809507
:1024E0009281892382830895FC01069622816213DA
:1024F00001C012823196E817F907C1F708952091BB
:1025000026012223C1F02091CE0127FF14C0262FDF
:102510002695269526952E3130F5FC01E20FF11D0A
:10252000677081E090E001C0880F6A95EAF79281B8
:10253000892B82830895FC0132962FEF30E0419180
:10254000641789F02F3F19F4411101C0232F3F5F19
:102550003630A9F72F3F39F0FC01E20FF11D27FDBE
:10256000FA956283089508952091C7013091C801BA
:102570002817390771F09093C8018093C701E09143
:10258000C501F091C601309721F00084F185E02D5E
:10259000099408952091C3013091C4012817390787
:1025A00071F09093C4018093C301E091C501F09153
:1025B000C601309721F00680F781E02D0994089537
:1025C000E091C501F091C601309721F00190F081B2
:1025D000E02D099480E008950F931F93CF93DF932C
:1025E000C42FD22FFC0182818823C9F04093C201FD
:1025F0000E9422129093C1018093C00180E28C0F4F
:10260000883008F057C0C77081E001C0880FCA95B4
:10261000EAF7DF91CF911F910F910C94DC1D80910F
:10262000C201481330C08091C0019091C1010E9445
:102630001312883C910538F510E21D0FCD17B9F043
:1026400080E28C0F883040F4C77081E001C0880FB1
:10265000CA95EAF70E94D51D183028F581E09D2F14
:10266000977001C0880F9A95EAF70E94DC1D802FB1
:102670000E940A1F1830F0F4D77081E001C0880F63
:10268000DA95EAF70AC080E28C0F883098F4C770B8
:1026900081E001C0880FCA95EAF7DF91CF911F91C1
:1026A0000F910C94D51D802FDF91CF911F910F9129
:1026B0000C940A1FDF91CF911F910F910895909173
:1026C000BB0190FF04C09695981740F003C081119C
:1026D00005C090E0961710F40C94C22561E00C94AC
:1026E0007E25882311F0FA0101C0FB010994609155
:1026F000BB01669570E04BE050E08CE091E00E94F9
:10270000FB28892B19F481E08093AB010E942212EF
:102710009093A5018093A40108958091BB0180FF4F
:102720000AC0869A81B38F7B91B390642FB7F894D7
:10273000EFEAF1E00BC0EFEAF1E0118210821282C1
:10274000339631E0EB3BF307C1F7EBCF31E0EB3BE6
:10275000F30789F0319148E091BB000000C037FFDA
:1027600081BB330F000000C000C000C081BB00C0AF
:102770004A9591F7EBCF2FBF8FE594E00197F1F7E2
:1027800000C000000895EF92FF920F931F93CF9324
:10279000DF938C01CFEAD1E0E12CF12CF8018481A8
:1027A000F2E0EF16F1041CF4882339F002C0811125
:1027B00004C09E014091BE0102C09E0140E06091B4
:1027C000BD018091BC010E94F6238FEFE81AF80A40
:1027D000239694E0E916F10409F70E948D13F8019D
:1027E000848190E00196817099278483DF91CF9155
:1027F0001F910F91FF90EF9008958F929F92AF924B
:10280000BF92CF92DF92EF92FF920F931F93CF93DD
:10281000DF93EC014C81042F10E09801D8010E9455
:10282000D2289B01AC010E94E8286B017C01E0E208
:10283000F0E0E01BF10BA5E5B0E09B01AC010E94CC
:10284000E8284B015C019F01DF010E94CA289B011F
:10285000AC010E94F3289B01AC012C0D3D1D4E1DC7
:102860005F1DC501B4010E94A228822FF22E99E2B9
:10287000921728F093E0299F900111240DC025E5BF
:1028800030E0281B3109C901880F991F280F391F13
:1028900037FF02C02F5F3F4F35952795122F1095B8
:1028A0009FEAC92E91E0D92E00E085E5E82EEF18C9
:1028B000802F869511F48E2D01C08F2D9601412F0A
:1028C0006091BD010E94F6230F5F83E0C80ED11C0A
:1028D000043071F70E948D138C81811102C091E048
:1028E00003C0803219F49FEF909319019091190160
:1028F000890F8C83DF91CF911F910F91FF90EF9003
:10290000DF90CF90BF90AF909F908F9008950F93DE
:102910001F93CF93DF93CFEAD1E0FE0111821082A3
:102920001282339681E0EB3BF807C1F700E010E03C
:102930008091AD01082E000C990B0817190794F02F
:1029400080911801082E000C990B8017910754F004
:102950009E014091BE016091BD018091BC010E9429
:10296000F62303C0198218821A820F5F1F4F239625
:1029700004301105E9F60E948D13809117019091A2
:10298000AD01980F9093AD0120911801280F20936D
:102990001801121614F493301CF0819580931701DE
:1029A000DF91CF911F910F910895CF92DF92EF9217
:1029B000FF920F931F93CF93DF93FC01828180FFDF
:1029C00003C0DD24DA9402C0DD24D394CFEAD1E041
:1029D00000E010E0198218821A8294E0E92EF12CAE
:1029E000C12C8091AC018C0D853014F0837002C035
:1029F00087FD8C5F082E000C990B0817190791F4BE
:102A00008091BE018E9DA0018F9D500D1124559582
:102A10004795559547959E016091BD018091BC01F8
:102A20000E94F623CD0CF1E0EF1AF108D1F60F5F0A
:102A30001F4F23960430110569F60E948D13809173
:102A4000AC0191E0D91206C0811102C083E006C03A
:102A5000815004C090E00196837099278093AC0167
:102A6000DF91CF911F910F91FF90EF90DF90CF906A
:102A70000895EF92FF921F93CF93DF93EC018FEABB
:102A8000E82E81E0F82E10E08C8197014091BE0184
:102A90006091BD01810F0E94F623115C83E0E80E76
:102AA000F11C1C3F89F70E948D139A818C8190FF45
:102AB00002C08F5F01C081508C83DF91CF911F9145
:102AC000FF90EF9008958091FA0187FF11C08091E7
:102AD000E80082FD05C08091F8018111F8CF11C096
:102AE0008091E8008B770BC08091F801882349F032
:102AF0008091E80080FFF8CF8091E8008E77809386
:102B0000E8000895982F973068F59093E90098179A
:102B100039F07091EC002091ED005091F00003C06D
:102B2000242F762F50E021FD02C09F5FECCF309123
:102B3000EB003E7F3093EB003091ED003D7F309312
:102B4000ED003091EB0031603093EB007093EC00BE
:102B50002093ED005093F0002091EE0027FDE5CF8B
:102B600080E008958F708093E90081E008952091BE
:102B70000002309101022617370748F061157105F0
:102B800039F42091E8002E772093E80001C0B901C4
:102B9000FC0120E06115710579F18091F80188232D
:102BA000F1F18530F1F18091E80083FD3CC0809126
:102BB000E80082FD2EC08091E80080FFEBCF2091DD
:102BC000F3008091F20090E0922B6115710551F0B5
:102BD0008830910538F421912093F10061507109FA
:102BE0000196F3CF21E0089709F020E08091E800FA
:102BF0008E778093E800CECF2111CFCF0AC080918D
:102C0000F801882361F0853061F08091E80083FD50
:102C10000AC08091E80082FFF2CF80E0089582E050
:102C2000089583E0089581E008950895BC0184E04B
:102C30000C946710BC0183E00C9467101F93CF9332
:102C4000DF93CDB7DEB7AA970FB6F894DEBF0FBEFD
:102C5000CDBFEAEFF1E08091F100819322E0E23014
:102C6000F207C9F78091FB01833009F461C030F4A9
:102C7000813071F0823009F49BC0B2C08A3009F40F
:102C800087C08B3009F46CC0893009F0A9C020C01E
:102C90008091FA01813A09F0A3C08091E800877F12
:102CA0008093E8008091FE019091FF01892B21F42F
:102CB00060E286ED91E003C060E080E090E070E0CB
:102CC0000E94B7158091E8008B778093E80088C058
:102CD0008091FA01813209F083C08091FE019091C8
:102CE000FF01029708F07CC08091E800877F809305
:102CF000E8008091E80082FD05C08091F801811113
:102D0000F8CF6EC02091F3008091F20090E0922BFA
:102D1000029731F48091F100813011F0863021F476
:102D20008091F1008093D5018091E8008B7754C0A9
:102D30008091FA01813A09F053C08091FE0190918F
:102D4000FF01892B09F04CC08091E800877F8093B8
:102D5000E8008091E80080FFFCCF8091260137C019
:102D60008091FA018132E1F58091FE019091FF019D
:102D7000892BB1F58091E800877F8093E8000E945D
:102D800063158091FC01809326010E94C01D28C01C
:102D90008091FA01813221F58091E800877F80934C
:102DA000E8000E9463158091FD018093D40118C052
:102DB0008091FA01813AA1F48091E800877F8093A5
:102DC000E8008091E80080FFFCCF8091D4018093DF
:102DD000F1008091E8008E778093E8000E946315EF
:102DE0008091E80083FFD9C18091FA019091FB01A5
:102DF000492F50E04A30510508F0CFC1FA01EE5991
:102E0000FF4F0C94C428803821F0823809F0C5C1E6
:102E100008C08091F6019091F701992389F08260B2
:102E20000FC08091FE018F70873008F0B6C180938B
:102E3000E9008091EB0085FB882780F91092E9007A
:102E40009091E800977F9093E8008093F1001092B2
:102E5000F10066C1282F2D7F09F09FC1882319F04A
:102E6000823061F09AC18091FC01813009F095C1F6
:102E7000933009F080E08093F7012EC08091FC012F
:102E800081112AC08091FE018F702FEF280F26300C
:102E900008F083C18093E9002091EB0020FF1CC063
:102EA000933021F48091EB00806214C09091EB008C
:102EB00090619093EB0021E030E0A90102C0440F43
:102EC000551F8A95E2F74093EA001092EA0080913C
:102ED000EB0088608093EB001092E9008091E8009D
:102EE000877F21C1811159C11091FC011F77809109
:102EF000E3008078812B8093E3008091E800877F56
:102F00008093E8000E9463158091E80080FFFCCF69
:102F10008091E30080688093E300111102C082E099
:102F200001C083E08093F80138C18058823008F0F6
:102F300034C18091FC019091FD018C3D53E09507D7
:102F400079F583E08A838AE289834FB7F894DE01BA
:102F5000139620E03EE051E2E32FF0E0509357005B
:102F6000E49120FF03C0E295EF703F5FEF708E2F7A
:102F700090E0EA3010F0C79601C0C0968D939D9303
:102F80002F5F243149F74FBF8091E800877F8093FE
:102F9000E8006AE270E0CE0101960E94B715AEC06B
:102FA0004091FE015091FF01292F33272330310535
:102FB000A9F068F42130310509F4FEC02230310552
:102FC00009F0EBC08FE990E0EDEBF3E044C0213273
:102FD000310521F12232310571F1DFC099278130AD
:102FE0009105A1F058F0029709F0D7C0EEE6F4E0A1
:102FF000E4918E2F90E0EEE6F4E02AC0E0EAF4E0FF
:10300000E4918E2F90E0E0EAF4E022C0EAE8F4E0F8
:10301000E4918E2F90E0EAE8F4E01AC041155105E2
:1030200009F4CFC04130510509F0B7C089E090E004
:10303000E8EEF3E010C04115510509F4C7C0413076
:10304000510509F0AAC086EB90E0E7ECF2E003C07E
:10305000009709F4A2C02091E800277F2093E800A0
:1030600020910002309101028217930708F49C011D
:1030700040E02115310589F18091F801882309F498
:103080003DC08530D9F18091E80083FD37C0809143
:10309000E80082FD2FC08091E80080FFEACF4091D8
:1030A000F3008091F20090E0942B2115310559F046
:1030B0008830910540F444914093F10031962150BD
:1030C00031090196F2CF41E0089709F040E0809184
:1030D000E8008E778093E800CCCF4111CDCF0AC0B5
:1030E0008091F801882351F0853041F08091E8000B
:1030F00083FD04C08091E80082FFF2CF8091E80058
:103100008B778093E80049C0803809F046C08091F1
:10311000E800877F8093E8008091F9018093F100B7
:103120008091E8008E778093E8000E94631535C097
:10313000811133C08091FC019091FD019927029784
:1031400064F58091E800877F8093E8001091FC018E
:103150001093F9010E946315111106C08091E300DC
:1031600087FD02C081E001C084E08093F80142E065
:1031700061EC81E00E94821542E261EC82E00E94F3
:10318000821542E361E883E00E94821542E361E830
:1031900084E00E9482158091F8018091E80083FF0D
:1031A0001AC08091E800877F8093E8008091EB004F
:1031B00080628093EB000FC082E190E0ECE5F4E0E8
:1031C0004ACF89E090E0EFECF3E045CF80E490E077
:1031D000EDE7F3E040CFAA960FB6F894DEBF0FBE3E
:1031E000CDBFDF91CF911F9108951F920F920FB61F
:1031F0000F9211242F933F934F935F936F937F937D
:103200008F939F93AF93BF93CF93DF93EF93FF93EE
:10321000C091E900CF708091EC00D82FD17080FD73
:10322000D0E81092E9008091F000877F8093F00051
:1032300078940E941E161092E9008091F000886038
:103240008093F000CD2BCF70C093E900FF91EF91F8
:10325000DF91CF91BF91AF919F918F917F916F91AE
:103260005F914F913F912F910F900FBE0F901F9044
:103270001895E8EDF0E080818E7F80831092E20067
:103280001092DA001092E100A0EEB0E08C91816023
:103290008C9380818F77808319BCA7EDB0E08C91EF
:1032A0008E7F8C9380818F7E80831092D3010895CE
:1032B000CF92DF92EF92FF920F931F93CF93DF9302
:1032C000C8EDD0E088818F7E8883E7EDF0E08081D3
:1032D0008160808384E082BF81E08093D301888114
:1032E0008E7F888302EE10E0F80110821092DA00DF
:1032F00081EEC82ED12CF601108288818F778883C9
:1033000088818068888388818F7D888319BC10922A
:10331000F8011092F9011092F7011092F60190EE67
:10332000E92EF12CF70180818B7F80838881816079
:10333000888342E060E080E00E948215F60180818F
:103340008E7F8083F80180818160808380818860A6
:103350008083F70180818E7F80838881806188836C
:10336000DF91CF911F910F91FF90EF90DF90CF9061
:1033700008951F920F920FB60F9211242F933F932F
:103380004F935F936F937F938F939F93AF93BF936D
:10339000EF93FF938091E10082FF09C08091E200EA
:1033A00082FF05C08091E1008B7F8093E1008091D6
:1033B000DA0080FF2AC08091D80080FF26C080916B
:1033C000DA008E7F8093DA008091D90080FF18C0E8
:1033D00080E189BD82E189BD09B400FEFDCF81E0B5
:1033E0008093F8018091D30181110FC00E94391997
:1033F0000E9458198091E20084608093E20005C029
:1034000019BC1092F8011092D3018091E10080FF65
:1034100017C08091E20080FF13C08091E2008E7F90
:103420008093E2008091E20080618093E2008091CD
:10343000D80080628093D80019BC85E08093F801A1
:103440008091E10084FF30C08091E20084FF2CC0B5
:1034500080E189BD82E189BD09B400FEFDCF809184
:10346000D8008F7D8093D8008091E1008F7E80937B
:10347000E1008091E2008F7E8093E2008091E20083
:1034800081608093E2008091F901882311F084E04B
:1034900007C08091E30087FD02C081E001C083E0A6
:1034A0008093F8018091F8018091E10083FF27C0AB
:1034B0008091E20083FF23C08091E100877F8093A9
:1034C000E10082E08093F8011092F9018091E1001F
:1034D0008E7F8093E1008091E2008E7F8093E200F6
:1034E0008091E20080618093E20042E060E080E051
:1034F0000E9482158091F00088608093F000FF9117
:10350000EF91BF91AF919F918F917F916F915F915B
:103510004F913F912F910F900FBE0F901F901895D4
:103520002091E4003091E50095E64091EC00842F75
:10353000817040FF23C08091E80080FD1DC0809114
:10354000F801882399F0853099F08091EB0085FD92
:1035500011C04091E4005091E5002417350729F38C
:10356000915011F09A01E1CF84E0089582E008952E
:1035700083E0089581E0089580E008954091E80097
:1035800042FFDDCF089580E090E00E94CA1280E003
:1035900090E00E94B412109280020E948A22E2E916
:1035A000F2E086E0DF011D928A95E9F710928C0225
:1035B00010928B0210928D020C94CC258F929F92C8
:1035C000AF92BF92EF92FF920F931F93CF93DF932F
:1035D0008090970190909801A0909901B0909A01E5
:1035E000409183025091840260918502709186021D
:1035F000842A952AA62AB72ACFE1D0E0E92EF12C19
:10360000082F10E0D501C4010C2E04C0B695A79573
:10361000979587950A94D2F780FD04C0219790F77B
:1036200080E016C0FE01EE0FFF1FEE0DFF1DEE0F36
:10363000FF1FEE0FFF1FE00FF11FEE0FFF1FEC55F6
:10364000FB4F859194910E946720019739F38C2F4D
:10365000DF91CF911F910F91FF90EF90BF90AF90AE
:103660009F908F900895CF93DF93D82FC92F0E94FA
:10367000DE1AEC2FF0E0E80FF11DE80FF11DEE0F60
:10368000FF1FEE0FFF1FED0FF11DEE0FFF1FEC559B
:10369000FB4F859194910E946720DF91CF9108950F
:1036A000FC01808191810E94331B92959F7096301E
:1036B00079F010F4925001C09A50923068F4803F33
:1036C00069F018F4883E40F409C0843F29F406C02C
:1036D000883E20F0813F11F080E0089581E0089558
:1036E0009F92AF92BF92CF92DF92EF92FF920F9391
:1036F0001F93CF93DF93CDB7DEB761970FB6F894E2
:10370000DEBF0FBECDBF8C0185E0F801DE011D9646
:1037100001900D928A95E1F7F801E28090912702DD
:103720006091280240912A0250912B0241155105C7
:1037300031F06F3F31F481E09F3F19F403C081E025
:1037400001C080E0F82FF1709F2E80FD1AC1F801B2
:1037500030812181C380D48087E2A82E82E0B82EF8
:10376000F0902902F601E41BF50BFF2009F4C6C016
:1037700080912C02E83CF10508F091C0482F407F71
:1037800009F050C0621311C093130FC0FE2CE1105A
:103790000CC08F70806180932C02C5010E9481044F
:1037A00080912C02F801858329C1CD2831F02F3F6B
:1037B00031F481E03F3F19F403C081E001C080E0B3
:1037C00080FD03C081E08E2502C080E090E0F82FEC
:1037D000F170FF2E80FF1CC080915E0240912D028F
:1037E00056E0841709F4E8C090E0589FF001599F13
:1037F000F00D1124E25DFD4F6181261306C060814A
:10380000631303C06281E61203C001968770E9CF9B
:10381000FE2CEE2009F4F2C080912C02816080938E
:103820002C0249C0621306C0931304C0E11002C009
:10383000F80186C0C8010E94501B882351F1EE2078
:1038400041F120912C02822F82958F7090E0029797
:1038500074F0809127029091280298878F831986AF
:10386000DB86CA862C87CE0107960E94810486E0FB
:10387000F801A7E2B2E001900D928A95E1F70E946B
:1038800023230AC06217C9F0C8010E94501B81118E
:103890001EC0C8010E948104FF24F394AFC0482FCA
:1038A000407F81F787E292E00E94810486E0F50183
:1038B00011928A95E9F7F12CA1C09313E5CFE1109D
:1038C000E3CFF8018583C8010E94810454C0EE2033
:1038D00001F320912C02822F82958F7090E0029745
:1038E00034F280912702909128029A8389831B8267
:1038F000DD82CC822E83CE010196B7CFE83CF10564
:10390000D0F5FE2CEE2029F2621327C0931325C0B8
:1039100020912C0220FD18C0822F82958F70482F95
:1039200050E04115510581F0F80125834F305105D4
:1039300041F08F5F982F9295907F822F8F70892B07
:103940008583C8010E94810486E0F801A7E2B2E005
:1039500001900D928A95E1F751C0C8010E94501B59
:10396000811185CF80912C02816080932C02C80147
:103970000E94810443C086E0F50111928A95E9F71F
:103980003DC0EE2009F485CFC8010E94501BF82EDF
:10399000882309F47ECF86E0F801A7E2B2E0019027
:1039A0000D928A95E1F780912702909128020E945A
:1039B000331B0E94232322C03D872E878D859E8541
:1039C0000E94331B292F22952F70223028F49F70DC
:1039D00039F0811105C00BC0243028F49F7049F4E0
:1039E000805E883020F0C8010E9481049F2CF92C51
:1039F00005C0F8019581907F99F7F9CF8F2D6196D9
:103A00000FB6F894DEBF0FBECDBFDF91CF911F91EF
:103A10000F91FF90EF90DF90CF90BF90AF909F906D
:103A20000895990F990F890F682F66956695669589
:103A3000982F977085E0689FB001112440E050E016
:103A400080E0FB01E40FF51FEE5FFD4F208130E0C9
:103A5000092E02C0369527950A94E2F72170332784
:103A6000042E01C0220F0A94EAF7822B4F5F5F4FAA
:103A70004530510531F70895990F990F890FE82FB7
:103A8000E695E695E695877051E001C0550F8A9559
:103A9000EAF785E0E89FF0011124EE5FFD4F20E09A
:103AA00030E070E04081CB01022E02C096958795F0
:103AB0000A94E2F781708195842785238427819376
:103AC0002F5F3F4F2530310569F7089560939701C7
:103AD000709398018093990190939A010C94C31A62
:103AE0000F931F9341E050E060E070E004C0440F8A
:103AF000551F661F771F8A95D2F7409550956095A0
:103B000070958091970190919801A0919901B09141
:103B10009A018A019B01082319232A233B23C90107
:103B2000B8011F910F910C94661D0F931F9341E0F4
:103B300050E060E070E004C0440F551F661F771F1F
:103B40008A95D2F78091970190919801A09199015F
:103B5000B0919A018A019B01082B192B2A2B3B2B30
:103B6000C901B8011F910F910C94661D60938302E7
:103B70007093840280938502909386020C94C31AFA
:103B80001092810280912601882331F08091CE012C
:103B900087FF02C08EE101C086E0E9E0F2E0DF01CC
:103BA0001D928A95E9F70C94C31A882321F00E948C
:103BB00083220C948A220895882339F090918102FF
:103BC000892B809381020C948A220895882309F41A
:103BD0005CC0823869F40E94E01281FF56C069E33C
:103BE00087E092E00E947F120E948A2269E30EC061
:103BF000833891F40E94E01280FF47C063E587E0BC
:103C000092E00E947F120E948A2263E587E092E0A0
:103C10000E9457120C948A22843869F40E94E012A0
:103C200082FF33C067E487E092E00E947F120E9427
:103C30008A2267E4EBCF9CEF980F913A10F4682F3B
:103C4000E5CF90E2980F983050F4877091E001C072
:103C5000990F8A95EAF7892F0E948322DBCF9BE593
:103C6000980F933020F480E090E00C94CA1298E50D
:103C7000980F973120F480E090E00C94B4128D3EC0
:103C800020F00E94F6250C94CC250895CF9388232C
:103C900009F4BEC0C82F8238B1F40E94E01281FD41
:103CA000B7C069E387E092E00E947F120E948A22F7
:103CB0002FEF81EE94E0215080409040E1F700C06A
:103CC000000069E317C08338E1F40E94E01280FD30
:103CD0009FC063E587E092E00E947F120E948A22E3
:103CE0002FEF81EE94E0215080409040E1F700C03A
:103CF000000063E587E092E00E945712CF910C9498
:103D00008A228438B1F40E94E01282FD81C067E407
:103D100087E092E00E947F120E948A222FEF81EEBC
:103D200094E0215080409040E1F700C0000067E43B
:103D3000E1CF8CEF8C0F813AC0F58091260188236A
:103D4000E1F08091CE0187FF18C0EC2FE695E69553
:103D5000E695F0E0E95FFD4F8281282F30E04C2F9F
:103D6000477081E090E002C0880F991F4A95E2F702
:103D700082239323892B61F412C0E9E0F2E08FE003
:103D800092E02191C21721F08E179F07D1F707C04B
:103D90006C2F87E092E00E9457120E948A226C2FBB
:103DA00087E092E00E947F12A9CF80E28C0F8830DA
:103DB00068F4C77081E090E001C0880FCA95EAF707
:103DC00090918102892B8093810298CFEBE5EC0FD3
:103DD000E33040F4F0E0E45CFE4F808190E0CF916E
:103DE0000C94CA12E8E5EC0FE73150F4F0E0EE0F66
:103DF000FF1FE15CFE4F80819181CF910C94B41242
:103E0000CD3E30F08C2F0E94AF26CF910C94CC2564
:103E1000CF9108951F93CF93DF93182F893319F013
:103E2000C0E0D0E002C0C0E5D0E0812F0E94461E75
:103E3000209741F08FE99FE00197F1F700C0000063
:103E40002197F6CF812FDF91CF911F910C94E61D22
:103E500080E008959091CE0192FF0DC0282F287127
:103E6000283019F4877F846006C0282F24712430FD
:103E700011F48B7F886093FF0DC0282F28712831A3
:103E800019F4877E846106C0282F2471243111F42F
:103E90008B7E88612091CF0120FF0DC0382F3871B3
:103EA000383019F4877F816006C0382F3171313086
:103EB00011F48E7F886021FF0DC0282F28712831D2
:103EC00019F4877E816106C0282F2171213111F4F8
:103ED0008E7E886194FD877E0895F894E82FE295A0
:103EE000EF70F0E031A1282F2F7081E090E001C049
:103EF000880F2A95EAF7982F9095932391A392A182
:103F0000892B82A3789408959F92AF92BF92CF920B
:103F1000DF92EF92FF920F931F93CF93DF9300D026
:103F2000CDB7DEB71A82198207E211E0AE014F5F0A
:103F30005F4F7A015A01CC24C394D12CF8018081BF
:103F40008F3F09F441C0F894E82FE295EF70F0E05C
:103F500021A18F70A60102C0440F551F8A95E2F778
:103F6000CA01922F982B91A392A18095892382A3B5
:103F7000789400C0E9E2F1E0912C31E021912F3FEB
:103F800089F0A22FA295AF70B0E090968C9190E04E
:103F90002F7002C0959587952A95E2F780FD02C0A3
:103FA000832F01C080E0982A330F51E0ED32F507EE
:103FB00029F7F80180818F3F11F00E946D1FF0EA10
:103FC000FA95F1F7F70190820F5F1F4FFFEFEF1A9D
:103FD000FF0A41E00932140709F0B0CF42E050E097
:103FE000B50185E991E00E940829FF24F394009728
:103FF00009F4F12C892B79F089819A8190939601AB
:104000008093950181E0809389020E94221290930F
:1040100088028093870280918902882391F08091A1
:104020008702909188020E941312059750F08091A8
:10403000950180939E018091960180939F0110923B
:10404000890280918A0291E0980F90938A028111EF
:104050002FC086E880937A0080EA80937B0080E41A
:1040600080937C0080917A00806480937A008091B4
:104070007A0086FDFCCF00917800909179008091C4
:104080007A008F7780937A0010E0192B83E01595E2
:1040900007958A95E1F700950F77E0919802F091E6
:1040A00099022EE342EB63E070E088E992E0099523
:1040B0008F2D0F900F90DF91CF911F910F91FF9057
:1040C000EF90DF90CF90BF90AF909F900895CF93E7
:1040D000DF938238910569F1B0F48133910509F4D9
:1040E0006FC048F48932910509F465C08A329105A0
:1040F00009F46BC08AC08533910509F457C0893330
:104100009105B9F082C0833E910571F138F4803E8B
:104110009105B1F0823E910511F177C0863E91057F
:10412000B9F1873E9105C9F1843E910509F06DC052
:1041300024C02091CE0120FD53C021FD51C065C097
:104140008091CE0180FD46C08091CF0180FF48C0A4
:104150008091CE0184FD50C183EE90E04FC18091EB
:10416000CE0182FF3AC0F4CF8091CE0182FD35C0EE
:104170008091CF0180FD34C0EBCF8091CF0181FFD2
:1041800035C08091CE0184FD37C187EE90E036C105
:104190008091CE0183FF27C0F4CF8091CE0183FDB3
:1041A00022C08091CF0181FD21C0EBCF8091CE0153
:1041B00085FD1FC021C08091CE0185FD1DC019C0A5
:1041C0008091CE0186FD1BC01DC08091CE0186FD71
:1041D00019C015C089E390E011C182EE90E00EC1D4
:1041E00080EE90E00BC186EE90E008C184EE90E096
:1041F00005C189E290E002C185E390E0FFC08AE258
:1042000090E0FCC081E390E0F9C0811531E59307AF
:1042100008F069C0811540E59407F0F09C0174E056
:10422000369527957A95E1F7922F9370482F437032
:1042300021E030E002C0220F331F4A95E2F73C68CC
:10424000392B982F9F709695969540E2949FC001C8
:104250001124822B932BD2C0883E910568F5803EB5
:10426000910508F0CBC0883A9105B8F4853A9105DC
:1042700048F0855AE82FF0E0E45CFE4F808190E042
:104280009064BCC08130910509F4B3C008F4B4C097
:104290008430910508F4B0C0B1C08F3B910508F09F
:1042A000ABC0885AE82FF0E0EE0FFF1FE15CFE4F35
:1042B000808191819464A2C0811520E2920758F414
:1042C000811531E0930708F099C08D3E910508F4FF
:1042D00093C0906593C0811540E4940708F48CC0A6
:1042E0009F70906A8BC0811525E5920708F042C047
:1042F000811534E5930728F0982F8827846F906AFA
:104300007DC0811543E59407B0F09C0123703327ED
:1043100041E050E002C0440F551F2A95E2F7282FD4
:104320002695269580E2289F90011124CA01822BB0
:10433000932B9A6863C0811522E5920728F4982F81
:104340008827816F906A5AC09C012370332741E00F
:1043500050E002C0440F551F2A95E2F7282F2695FA
:10436000269580E2289F90011124CA01822B932B6D
:104370009C6844C0EC01811539E59307A8F48115C8
:10438000984528F09C2F8827806F906A37C0C11508
:1043900086E5D80788F58C2F0E942A1F8F7190E040
:1043A000982F882790622AC081152AE5920790F4F9
:1043B0008C2F8F700E942A1F94E0D695C7959A95EE
:1043C000E1F7CF70D0E0DC2FCC27D0699E01282BFD
:1043D000C90114C090568115904270F48D2F8F71D1
:1043E0000E942A1F282F2F71CE0199279062922BAD
:1043F00005C081E090E002C080E090E0DF91CF91C5
:104400000895CF9384E090E00E943228C82F82E282
:1044100090E00E9432282C2F30E0A901582BCA01CD
:10442000CF91089569EE7EEF80E090E00E946428CD
:1044300060E082E090E00E94462860E083E090E047
:104440000E944628109283021092840210928502E4
:104450001092860260E084E090E00E94462860E0CE
:1044600082E290E00E94462860E085E090E00E94B1
:10447000462860E086E090E00E9446286FEF87E0E3
:1044800090E00E94462840E050E0BA0188E090E0C9
:104490000E94582860E08DE090E00E94462840E0AD
:1044A00050E0BA0188E190E00E94582860E087E17E
:1044B00090E00E94462840E050E0BA018CE190E094
:1044C0000E94582860E070E080E290E00E9464283A
:1044D00040E050E0BA0188E190E00E94582840E0B6
:1044E00050E0BA018FE090E00E94582840E050E090
:1044F000BA0183E190E00C945828809182028111E6
:104500001092820208958095909181028923809370
:10451000810208959091810280918002982B90935E
:104520000702809182028823D9F0892B80930702A9
:1045300080912601882331F08091CE0187FF02C04F
:104540008EE101C086E0E9E0F2E090E0815028F0E1
:1045500021912223D9F39F5FF9CF91110E947D22EF
:1045600040E250E060E672E087E092E00E940829B5
:10457000892B21F180E2E7E0F2E0A0E6B2E00190D1
:104580000D928A95E1F7E091C501F091C60130974F
:10459000A9F080912601882359F08091CE0187FFF0
:1045A00007C0809107028093080286E0809307028B
:1045B0000280F381E02D87E092E009940895209134
:1045C0005F028095822380935F02982F977099F401
:1045D00030E0482F082E000C550B2417350759F0F2
:1045E0009091CF0192FD07C08595859585950E9494
:1045F000701D10925F020895CF93C091CF01C2FB4E
:10460000992790F9981799F080FBC2F9C093CF01D0
:104610006091CE0184E090E00E9446286C2F82E2F7
:1046200090E00E94462882E0CF910C94DF22CF9147
:10463000089580915E0290912D02891719F08F5F85
:104640008770FBCF08950F931F93CF93DF938091D3
:104650002C0282958F7009F05DC080912902882319
:1046600009F458C080915E0210912D0260912702DA
:1046700070912802C0912A02D0912B0291E06F3FE5
:1046800009F090E0292F06E0811709F443C0209734
:1046900021F07F3F21F030E003C031E001C0322F34
:1046A00090E030FD34C0089FF001099FF00D112407
:1046B000DF01A25DBD4F11963C911197371327C0C2
:1046C0003C91361324C012963C91129731111FC0B1
:1046D00013964D915C9114974C1B5D0B483C510512
:1046E000B0F480912C028F70806180932C02ED5C7D
:1046F000FD4F80818F708061808387E292E00E940D
:104700008104DF91CF911F910F910C941923019691
:104710008770BACFDF91CF911F910F91089590913B
:10472000BB0190FF0CC0EFEAF1E08183608342831C
:10473000339691E0EB3BF907C1F70C948D13089584
:104740008091BB01282F269530E02115310519F401
:104750008170826005C02532310524F08170886443
:104760008093BB010895CF92DF92EF92FF926B018D
:104770007C010E94A023B701A60188E090E0FF9091
:10478000EF90DF90CF900C9458288091BF01882340
:1047900019F081508093BF016091BB017091BC0101
:1047A0008091BD019091BE010C94B3238091BF0113
:1047B000833018F48F5F8093BF016091BB017091CB
:1047C000BC018091BD019091BE010C94B323EBEB31
:1047D000F1E083E0808311828FEF828383831482F0
:1047E00060817181828193810C94B323AF92BF92D7
:1047F000CF92DF92EF92FF920F931F93CF93DF93AD
:10480000E82EF62EE901E42FF0E0611106C0EC522B
:10481000FB4FE4914E2F2E2F71C0062F10E0EC526B
:10482000FB4F4491F42FC42ED12C26E0829FC0016F
:1048300011242FEF30E0B9010E947A285BEA560379
:10484000C001579F900D11248E0D911D8E0D911D4D
:10485000582F550F580FD901A01BB10BAC9DC001AB
:10486000AD9D900DBC9D900D1124E92FF59ED001BA
:104870001124AB2FBB277901EA1AFB0AEC9CD0016B
:10488000ED9CB00DFC9CB00D11245901A51AB10886
:10489000A09E7001A19EF00CB09EF00C1124EF2C94
:1048A000FF242E193F092C9D80012D9D100D3C9D4C
:1048B000100D1124212F6230710591F048F461151B
:1048C0007105E1F061307105B9F4242F4B2F16C04A
:1048D0006430710569F040F06630710579F00CC004
:1048E000242F492FE12F0AC0492FEF2F2B2F06C06D
:1048F000292FE42F412F02C0292FEB2F4983288332
:10490000EA83DF91CF911F910F91FF90EF90DF909D
:10491000CF90BF90AF900895CF93DF9300D01F92B8
:10492000CDB7DEB79091BB0190FF0AC09E012F5F0B
:104930003F4F0E94F6234B8169818A810E948F2319
:104940000F900F900F90DF91CF9108957F928F92EB
:104950009F92AF92BF92CF92DF92EF92FF920F930E
:104960001F93CF93DF9300D01F92CDB7DEB7182FE0
:10497000D62E042FC22E9091BB0190FF6CC0E92F60
:10498000E695AE2FB0E0A359BE4F8C918093AA015B
:104990009E7F923061F49E012F5F3F4F812F0E94D6
:1049A000F6234B8169818A810E948F2342C0823025
:1049B00019F40091BE013DC0863019F41091BC017C
:1049C00038C08930D9F38931A1F5E9512E2F2170F2
:1049D000722EE695F0E0EC52FA4F859094903FEA03
:1049E000A32E31E0B32EE12CF12C99248E9CC00132
:1049F0008F9C900D9E9C900D112496958795969571
:104A00008795711002C0810F03C0212F281B822FB0
:104A10009501402F6D2D0E94F6238FEFE81AF80ABA
:104A200023E0A20EB11C84E0E816F104F9F60E941E
:104A30008D131093BC01D092BD010093BE01CC2018
:104A400051F06091BB017091BC018091BD019091CA
:104A5000BE010E94B3230F900F900F90DF91CF9172
:104A60001F910F91FF90EF90DF90CF90BF90AF908C
:104A70009F908F907F900895EBEBF1E0438128E0C9
:104A8000421B08F440E021E0628181810C94A6245D
:104A9000EBEBF1E0438128E0420F08F44FEF21E017
:104AA000628181810C94A624EBEBF1E0628128E025
:104AB000621B08F460E021E0438181810C94A6240C
:104AC000EBEBF1E0628128E0620F08F46FEF21E088
:104AD000438181810C94A624EBEBF1E0818121E0FC
:104AE0004381628188500C94A624EBEBF1E0818134
:104AF00021E043816281885F0C94A6249091BB01E0
:104B000090FF36C09170811102C0926006C085325C
:104B100010F0986402C0880F982B9093BB01662315
:104B200051F06091BB017091BC018091BD019091E9
:104B3000BE010E94B3236091BB01669570E04BE01B
:104B400050E08CE091E00E94FB28892B19F0109234
:104B5000AB0102C00E94771381E08093A70120E09F
:104B60004091BE016091BD018091BC010C94A624CE
:104B700008958091BB018695815009F484E261E03B
:104B80000C947E258091BB0186958F5F853208F05D
:104B900081E061E00C947E250E9422122091940213
:104BA000211104C020919502222321F090939102BB
:104BB0008093900220919602211104C020919702C7
:104BC000222321F090938F0280938E02E091C50101
:104BD000F091C601309749F082E080939202048000
:104BE000F581E02D82E992E0099408958D3E39F433
:104BF0009091950297FF35C01092950259C08E3E54
:104C000029F4909195021916BCF32BC0909194024F
:104C10008F3E29F497FF25C01092940249C0803F2F
:104C200019F41916CCF31DC090919602893F29F40E
:104C30001916BCF4109296023BC08A3F19F497FFF4
:104C400010C0F8CF8B3F39F49091970297FF09C0BD
:104C5000109297022DC08C3F21F490919702191663
:104C6000BCF39FE0980F983080F421E030E0A90178
:104C700002C0440F551F9A95E2F7CA0180959091A2
:104C8000930289238093930213C08D3F21F4809176
:104C90008D028E7F0BC08E3F21F480918D028D7F1F
:104CA00005C08F3F29F480918D028B7F80938D0208
:104CB00080919402811106C080919502811102C0F9
:104CC00010928C0280919602811106C08091970209
:104CD000811102C010928B02089580918D0280FD97
:104CE00016C081FD16C082FD18C080918B028823FA
:104CF00091F0883290F428E0829FC001112468E28C
:104D000070E00E948E28862F672B29F007C082E072
:104D1000089584E0089581E0089588E008958091E1
:104D20008D0280FD14C081FD14C082FD16C08091EB
:104D30008C02882381F08E3180F420E5829FC001AF
:104D400011246EE170E00E948E28862F089584E180
:104D5000089588E2089588E0089580E508958D3EDD
:104D600021F40E948F26819504C08E3E29F40E9472
:104D70008F268093950208958F3E21F40E948F26FE
:104D8000819504C0803F29F40E948F26809394026D
:104D90000895893F19F40E946D2605C08A3F31F4B9
:104DA0000E946D2681958093960208958B3F21F491
:104DB0000E946D26819504C08C3F29F40E946D26C7
:104DC0008093970208959FE0980F983078F421E03F
:104DD00030E0A90102C0440F551F9A95E2F7CA01BD
:104DE00090919302892B8093930208958D3F21F433
:104DF00080918D0281600BC08E3F21F480918D02E5
:104E0000826005C08F3F29F480918D028460809379
:104E10008D020895CF92DF92EF92FF920F931F932E
:104E2000CF93DF9300D01F92CDB7DEB77C01162F52
:104E3000D42EC22E8091BD028430F9F4E091B202EA
:104E4000F091B302309709F4B7C0C701019763E04E
:104E500070E00E947A28CB01880F991F860F971F58
:104E600019834A83CB824E2D481B9E012F5F3F4FF3
:104E7000BC0188E992E00995ACC082E0E816F10433
:104E800009F44FC083E0E816F10431F081E0E81640
:104E9000F10409F08DC078C0862F807F803AE1F060
:104EA00050F48038A1F0803909F086C0E0919C026E
:104EB000F0919D0225C0803EA1F0803FB9F0803B7B
:104EC00009F07AC0E0919A02F0919B0219C0E0913A
:104ED0009E02F0919F0214C0E091A002F091A10205
:104EE0000FC0E091A202F091A3020AC0623F09F054
:104EF00063C0E091A402F091A502309731F45CC048
:104F0000309709F459C0123F21F42C2D4D2D62EF3A
:104F100004C02C2D4D2D612F6F7088E992E009950A
:104F200058C0862F807F803D51F0803F69F0803CE3
:104F300009F042C0E091A602F091A70215C0E091ED
:104F4000A802F091A90210C0633F29F4E091AA02DF
:104F5000F091AB0206C0613F79F5E091AC02F091AF
:104F6000AD02309739F428C0309731F1812F8D7F11
:104F7000813F19F44D2D612F03C04D2D612F6F70AE
:104F800088E992E0099525C0683F28F0E091AE02DB
:104F9000F091AF0206C0663F79F4E091B002F09163
:104FA000B102309749F0612F88E992E0099511C06C
:104FB00084E0E816F104D8F4E091B402F091B5026F
:104FC000309739F00C2D2D2D412FB70188E992E053
:104FD0000995E091B602F091B702309759F00C2D87
:104FE0002D2D412FB70188E992E0099503C0E12CEE
:104FF000F12CE2CF0F900F900F90DF91CF911F9186
:105000000F91FF90EF90DF90CF900895EF92FF9275
:105010000F931F93CF93DF937C018B010E94901A13
:10502000811119C0E70101151105A1F08091E80077
:1050300085FD0AC08091E8008E778093E8000E9489
:10504000901A882381F307C089918093F100015061
:105050001109E9CF80E0DF91CF911F910F91FF906F
:10506000EF900895F999FECF92BD81BDF89A9927E6
:1050700080B50895A6E1B0E044E050E00C946C28BF
:10508000A8E1B0E042E050E00C946C28262FF9999A
:10509000FECF92BD81BDF89A019700B4021639F097
:1050A0001FBA20BD0FB6F894FA9AF99A0FBE089568
:1050B0000396272F0E9447280E944628252F0E94EA
:1050C0004728242F0C9447280196272F0E94472811
:1050D0000C944628DC01CB01FC01F999FECF06C0F7
:1050E000F2BDE1BDF89A319600B40D9241505040A6
:1050F000B8F70895AA1BBB1B51E107C0AA1FBB1F2D
:10510000A617B70710F0A61BB70B881F991F5A9553
:10511000A9F780959095BC01CD01089597FB072EC6
:1051200016F4009407D077FD09D00E947A2807FC76
:1051300005D03EF4909581959F4F089570956195A7
:105140007F4F0895A1E21A2EAA1BBB1BFD010DC0C3
:10515000AA1FBB1FEE1FFF1FA217B307E407F50727
:1051600020F0A21BB30BE40BF50B661F771F881F03
:10517000991F1A9469F760957095809590959B0199
:10518000AC01BD01CF010895EE0FFF1F0590F49112
:10519000E02D09940E94D228332312F48A1B9B0B22
:1051A0000C94E328A29FB001B39FC001A39F700D90
:1051B000811D1124911DB29F700D811D1124911D1F
:1051C00008950E94D228B7FF0895821B930B08957B
:1051D0000E94D228A59F900DB49F900DA49F800D92
:1051E000911D11240895B7FF0C94E8280E94E82827
:1051F000821B930B0895FC014150504030F0019008
:105200000616D1F73197CF01089588279927089579
:10521000FB01DC0104C08D910190801921F4415003
:0E5220005040C8F7881B990B0895F894FFCFF3
:10522E009D0FC20FA30F1A161616151601191A1B6B
:10523E001C1D1E1F202122010201038340000001BC
:10524E0004400000010001F0F1303132330203025C
:10525E00000001000101010101000101818283E2D0
:10526E0000E900EA00B500B600B700CD008301CC1E
:10527E00008A0192019401210223022402250226B2
:10528E000227022A02B300B4006F00700000010270
:10529E000202020606060909090909090F0F0F0F76
:1052AE000F0F151515181919191919191919191981
:0252BE002324A7
:00000001FF
